:1000000001308A008F2900002310F6327210F3327B
:100010007110203AE536F02DED255D10E83AED2F10
:10002000F4326D38DB36CB2E2034F536DB12A52EBC
:100030002000E230F22FF4326D38DB36CB2E203840
:10004000F232F3397539E52D6828E12E2010413759
:10005000E536EF2D7036F317F32E6334E531EB06FA
:100060008A060A006608E8006508E7006808FA00E2
:100070006708840083137A188317800803194428BB
:10008000E70A0319E80A362865086702F7006808D6
:10009000FA006608031C660FFA027708F8000800E9
:1000A00083168613831286130830F8005728000041
:1000B000F8176828F813E90C03188617031C861331
:1000C000781768287813F80B5B28662800008617D5
:1000D0003F308400840B6A280000F81B5A28781BE4
:1000E000622808002430B3004930B4006430B50001
:1000F0003A30B6002030B7006D30B8006130B9003A
:100100006930BA006E30BB002E30BC006330BD00D9
:100110002030BE003230BF003830C0003530C10062
:100120003830C2002030C3003230C4003030C50047
:100130003130C6003330C7002D30C8003030C90020
:100140003330CA002D30CB003230CC00CD0020300F
:10015000CE003130CF003630D0003A30D1003030D0
:10016000D2003430D3003A30D4003130D5003330AF
:10017000D6005A30D7002030D8006B30D90061301B
:10018000DA006B30DB006C30DC006930DD006B3096
:10019000DE002030DF002430E000E101E6013330F2
:1001A000E500322001307802333E840083130008DA
:1001B000243C031DE528E6013330E5003220013000
:1001C0007802333E840083138001043003178D00CE
:1001D00000308F00031025300313E500831603174A
:1001E0008C170C140000000003181D2983120C0842
:1001F0007F390313E60003170D080313E700031705
:100200000F080313E8006608E90050206708031789
:100210008D000313680803178F0083168C170C14C6
:100220000000000083120313E50B17291A29831617
:1002300003171D293C298316031783120C0D0E0D7D
:100240007F390313E60003170D080313E7000317B4
:100250000F080313E8006608E90050206708031739
:100260008D000313680803178F008D0A03198F0A86
:1002700003100313E50BEE282530E90050205D3014
:10028000E90050202030E9005020193003178D007C
:1002900000308F0083168C170C14000000008312AE
:1002A0000C087F3903198B290313E50003170D0888
:1002B0000313E60003170F080313E7006508E900BE
:1002C0005020660803178D000313670803178F007B
:1002D00083168C170C140000000083120C0D0E0DF9
:1002E0007F3903198B290313E50003170D08031346
:1002F000E60003170F080313E7006508E900502024
:10030000660803178D000313670803178F008D0A13
:1003100003198F0A4A2903138A110A12032A840136
:1003200083131F308305713083168F000F088613E7
:1003300083128617831603170908C039890003132F
:100340001F129F1200300317880083128701880153
:1003500089010313A001A101FF30B200713083169F
:100360008F000F0809308312031785000F30F70044
:10037000031381018130840083130008F0390738AA
:10038000800064000008F739F719F039770480001D
:100390006400831603170908C039890003131F126C
:1003A0009F12003003178800831203131F139F133B
:1003B00083169F1383121F1483160108C739283828
:1003C00081003530831290000030F8009200003038
:1003D0008316920083123215320883168700831227
:1003E000970183169B019C0101309D008312031726
:1003F00087018801890103133211320883168700AF
:08040000831207157228630046
:04400E00F52CFF3F4F
:00000001FF
